 adpinv

 Timestamp is 4a76a358 (Mon Aug 03 14:14:08 2009)

 Preferred load address is 0000000000010000

 Start         Length     Name                   Class
 0001:00000000 000238b9H .text                   CODE
 0001:000238c0 000000d1H .text$s                 CODE
 0002:00000000 000000b8H .idata$5                DATA
 0002:000000c0 0000001cH .rdata                  DATA
 0002:000000dc 00000051H .rdata$debug            DATA
 0002:00000130 000009bcH .xdata                  DATA
 0003:00000000 000008e0H .data                   DATA
 0003:000008e0 00000280H .bss                    DATA
 0004:00000000 00000fe4H .pdata                  DATA
 0005:00000000 00000061H INIT                    CODE
 0005:00000064 00000028H .idata$2                CODE
 0005:0000008c 00000014H .idata$3                CODE
 0005:000000a0 000000b8H .idata$4                CODE
 0005:00000158 00000214H .idata$6                CODE
 0006:00000000 000000a0H .rsrc$01                DATA
 0006:000000a0 00000b90H .rsrc$02                DATA

  Address         Publics by Value              Rva+Base               Lib:Object

 0000:00000000       ___safe_se_handler_table   0000000000000000     <absolute>
 0000:00000000       ___safe_se_handler_count   0000000000000000     <absolute>
 0001:00000008       WriteEvent                 0000000000011008 f   win_utils.obj
 0001:00000054       RtlUnicodeStringCbCatN     0000000000011054 f i regreader.obj
 0001:00000174       readRegConfiguration       0000000000011174 f   regreader.obj
 0001:0000043c       SP_INC                     000000000001143c f   ntinit.obj
 0001:000004dc       DriverEntry                00000000000114dc f   ntinit.obj
 0001:000006c4       HwFindAdapter              00000000000116c4 f   ntinit.obj
 0001:00000df8       HwAdapterControl           0000000000011df8 f   ntinit.obj
 0001:00000eb4       OsmTimer                   0000000000011eb4 f   ntinit.obj
 0001:0000106c       HwInitialize               000000000001206c f   ntinit.obj
 0001:000011d0       HwStartIo                  00000000000121d0 f   ntinit.obj
 0001:00001a88       HwBuildIo                  0000000000012a88 f   ntinit.obj
 0001:00001b94       HwIoIsr                    0000000000012b94 f   ntinit.obj
 0001:00001c18       HwResetBus                 0000000000012c18 f   ntinit.obj
 0001:00001c40       PostIOD                    0000000000012c40 f   ntinit.obj
 0001:000020dc       DeQueueIOD                 00000000000130dc f i ntinit.obj
 0001:000021a8       OsmGetIoTimeoutTicks       00000000000131a8 f i ntinit.obj
 0001:000022d4       OsmSetCustomIOStatus       00000000000132d4 f i ntinit.obj
 0001:00002408       OsmCompleteSrb             0000000000013408 f i ntinit.obj
 0001:00002598       AdjustTimeout              0000000000013598 f   ntinit.obj
 0001:000026ac       PostOsmResetTMF            00000000000136ac f   ntinit.obj
 0001:00002844       PostOsmTMF                 0000000000013844 f   ntinit.obj
 0001:00002958       OsmTMFEvents               0000000000013958 f   ntinit.obj
 0001:00002bec       XReturnPhysAddr            0000000000013bec f   osif.obj
 0001:00002c4c       XMemZero                   0000000000013c4c f   osif.obj
 0001:00002cb0       XMemCpy                    0000000000013cb0 f   osif.obj
 0001:00002cf4       XMicrosecondDelay          0000000000013cf4 f   osif.obj
 0001:00002d48       XNotify                    0000000000013d48 f   osif.obj
 0001:00002e98       XAlignedMemAllocPastOH     0000000000013e98 f   osif.obj
 0001:00002ed0       OSMMapIOHandle             0000000000013ed0 f   osmif.obj
 0001:00002f6c       OSMReleaseIOHandle         0000000000013f6c f   osmif.obj
 0001:00002f7c       OSMAdjustBusAddress        0000000000013f7c f   osmif.obj
 0001:00002f88       OSMReadUExact8             0000000000013f88 f   osmif.obj
 0001:00002fac       OSMReadUExact16            0000000000013fac f   osmif.obj
 0001:00002fd0       OSMReadUExact32            0000000000013fd0 f   osmif.obj
 0001:00002ff0       OSMReadStringUExact8       0000000000013ff0 f   osmif.obj
 0001:0000303c       OSMReadStringUExact16      000000000001403c f   osmif.obj
 0001:00003088       OSMReadStringUExact32      0000000000014088 f   osmif.obj
 0001:000030d4       OSMWriteUExact8            00000000000140d4 f   osmif.obj
 0001:000030f8       OSMWriteUExact16           00000000000140f8 f   osmif.obj
 0001:00003120       OSMWriteUExact32           0000000000014120 f   osmif.obj
 0001:00003144       OSMWriteStringUExact8      0000000000014144 f   osmif.obj
 0001:00003194       OSMWriteStringUExact16     0000000000014194 f   osmif.obj
 0001:000031f4       OSMWriteStringUExact32     00000000000141f4 f   osmif.obj
 0001:00003250       OSMReadPCIConfigurationDword 0000000000014250 f   osmif.obj
 0001:00003264       OSMReadPCIConfigurationWord 0000000000014264 f   osmif.obj
 0001:000032f4       OSMReadPCIConfigurationByte 00000000000142f4 f   osmif.obj
 0001:00003384       OSMWritePCIConfigurationDword 0000000000014384 f   osmif.obj
 0001:000033c8       OSMWritePCIConfigurationWord 00000000000143c8 f   osmif.obj
 0001:0000340c       OSMWritePCIConfigurationByte 000000000001440c f   osmif.obj
 0001:00003450       OSMWriteEventLog           0000000000014450 f   osmif.obj
 0001:00003474       FillOutOSMPointers         0000000000014474 f   osmif.obj
 0001:00003608       RetryIODDispatch           0000000000014608 f   resource.obj
 0001:00003654       AssignDMASenseBuffer       0000000000014654 f   resource.obj
 0001:000036c0       CreateSpecialIODs          00000000000146c0 f   resource.obj
 0001:00003798       AllocStruc                 0000000000014798 f   resource.obj
 0001:00003888       InitIOB                    0000000000014888 f   resource.obj
 0001:000038ec       InitSpecialIOB             00000000000148ec f   resource.obj
 0001:00003aa4       AllocIODs                  0000000000014aa4 f   resource.obj
 0001:00003b30       InitIOD                    0000000000014b30 f   resource.obj
 0001:00003bb8       GetFreePhysDevice          0000000000014bb8 f   resource.obj
 0001:00003c28       GetFreeTSCB                0000000000014c28 f   resource.obj
 0001:00003cb4       AllocSpecialIODs           0000000000014cb4 f   resource.obj
 0001:00003d08       Res_InitAndRebuildIODLink  0000000000014d08 f   resource.obj
 0001:00003e04       PhysPolledIo               0000000000014e04 f   physif.obj
 0001:00004018       PostPhysQueueQuiesce       0000000000015018 f   physif.obj
 0001:00004144       PhysQueueEnablePhy         0000000000015144 f   physif.obj
 0001:0000427c       PostStopPhysQueueEnablePhy 000000000001527c f   physif.obj
 0001:000042b8       PostPhysQueueEnablePhy     00000000000152b8 f   physif.obj
 0001:000045a8       PhysGetDevicePortTSH       00000000000155a8 f   physif.obj
 0001:00004ba0       PhysGetLuTSH               0000000000015ba0 f   physif.obj
 0001:00004e28       CdaCreatePD                0000000000015e28 f   physif.obj
 0001:00004f68       PhysAddSasDevice           0000000000015f68 f   physif.obj
 0001:00005290       PhysRemoveSasDevice        0000000000016290 f   physif.obj
 0001:000053e8       CdaFreeSDPD                00000000000163e8 f   physif.obj
 0001:000054a4       CdaRemoveExistingDevice    00000000000164a4 f   physif.obj
 0001:00005554       PhysStartAdapter           0000000000016554 f   physif.obj
 0001:00005844       InitializeSasChim          0000000000016844 f   physif.obj
 0001:00005acc       SizeIOBMemNeed             0000000000016acc f   physif.obj
 0001:00005b64       ValidatePort               0000000000016b64 f   physif.obj
 0001:00005c78       HandlePortEvents           0000000000016c78 f   physif.obj
 0001:00006040       OSMPortEvent               0000000000017040 f   physif.obj
 0001:000060d0       ProcessNewTargets          00000000000170d0 f   physif.obj
 0001:00006280       IssueTestDevicePresentSequence 0000000000017280 f   physif.obj
 0001:0000635c       PostTestDevicePresent_InitializationTime 000000000001735c f   physif.obj
 0001:00006424       ValidateTargetsForPort     0000000000017424 f   physif.obj
 0001:000066dc       PostDevicePortInitialization 00000000000176dc f   physif.obj
 0001:00006884       PerformDevicePortInitialization 0000000000017884 f   physif.obj
 0001:00006a58       PerformLuDiscovery         0000000000017a58 f   physif.obj
 0001:00006c30       PostProbeLuForSasDevice    0000000000017c30 f   physif.obj
 0001:00006e90       PostPacForPort             0000000000017e90 f   physif.obj
 0001:00007040       PostPacForAdapter          0000000000018040 f   physif.obj
 0001:000071a8       CheckForNewDevicePorts     00000000000181a8 f   physif.obj
 0001:00007200       OSMAdapterEvent            0000000000018200 f   physif.obj
 0001:000072e4       HandleAdapterEvents        00000000000182e4 f   physif.obj
 0001:00007924       DiscoverNewPorts           0000000000018924 f   physif.obj
 0001:00007a74       OSMLuEvent                 0000000000018a74 f   physif.obj
 0001:00007aa4       HandleLuEvents             0000000000018aa4 f   physif.obj
 0001:00007d34       PostCdaPerformLuRecovery   0000000000018d34 f   physif.obj
 0001:00007ee8       PostCdaAbortTaskSet        0000000000018ee8 f   physif.obj
 0001:000080a8       OSMIobEvent                00000000000190a8 f   physif.obj
 0001:00008208       AbortTaskForProbeLuComplete 0000000000019208 f   physif.obj
 0001:00008244       CdaStopAdapter             0000000000019244 f   physif.obj
 0001:0000857c       CdaRestartAdapter          000000000001957c f   physif.obj
 0001:000085e0       ConvertAddressToBytes      00000000000195e0 f   physif.obj
 0001:0000861c       SaveCrashdumpPtrs          000000000001961c f   physif.obj
 0001:00008704       CheckPendingPhysDeviceRemval 0000000000019704 f   physif.obj
 0001:0000883c       PostEnableFailedPhyDone    000000000001983c f   physif.obj
 0001:000088e8       CheckFailedPhyBitMask      00000000000198e8 f   physif.obj
 0001:00008a74       PostResetPortDone          0000000000019a74 f   physif.obj
 0001:00008b90       HandleLocalLuEvents        0000000000019b90 f   physif.obj
 0001:00008c08       CdaLuValidationToPort      0000000000019c08 f   physif.obj
 0001:00008c68       CdaDeviceLuValidation      0000000000019c68 f   physif.obj
 0001:00008e34       CdaDeviceLuValidationComplete 0000000000019e34 f   physif.obj
 0001:000092a0       RestoreCrashDumpPointers   000000000001a2a0 f   physif.obj
 0001:00009368       GetAndSetCHIMConfiguration 000000000001a368 f   physif.obj
 0001:00009444       AllocateCHIMMemory         000000000001a444 f   physif.obj
 0001:000095c4       CdaStartScan               000000000001a5c4 f   core.obj
 0001:00009614       AddIODToIOQueue            000000000001a614 f   core.obj
 0001:00009660       RemoveIODFromIOQueue       000000000001a660 f   core.obj
 0001:000096a0       ResetAdapter               000000000001a6a0 f   core.obj
 0001:00009854       ResetHardware              000000000001a854 f   core.obj
 0001:00009934       ResetHardwareComplete      000000000001a934 f   core.obj
 0001:00009994       ResetAdapterComplete       000000000001a994 f   core.obj
 0001:00009a28       LockAdapterBuffer          000000000001aa28 f   core.obj
 0001:00009a94       ResetLogicalUnit           000000000001aa94 f   core.obj
 0001:00009bf8       ResetDevicePort            000000000001abf8 f   core.obj
 0001:00009db0       ResetDevicePortComplete    000000000001adb0 f   core.obj
 0001:0000a044       SetupPollIOD               000000000001b044 f   core.obj
 0001:0000a2f4       ResetLogicalUnitComplete   000000000001b2f4 f   core.obj
 0001:0000a3b4       ExecuteOSCommand           000000000001b3b4 f   core.obj
 0001:0000a42c       XCfgDiscoveryOnlyIF        000000000001b42c f   core.obj
 0001:0000a454       PostXCfgDiscoveryOnlyIF    000000000001b454 f   core.obj
 0001:0000a4c8       PhysDeviceMemoryAllocation 000000000001b4c8 f   core.obj
 0001:0000a584       GetCHIMMemoryRequirement   000000000001b584 f   core.obj
 0001:0000a764       RestartPendingIOs          000000000001b764 f   core.obj
 0001:0000a800       PostPendingIODs            000000000001b800 f   core.obj
 0001:0000a9b4       CdaTimer                   000000000001b9b4 f   core.obj
 0001:0000acd4       PostATAPICommand           000000000001bcd4 f   core.obj
 0001:0000ae7c       SpecialMemoryAllocation    000000000001be7c f   core.obj
 0001:0000b110       CdaTMFRequest              000000000001c110 f   core.obj
 0001:0000b29c       PollInformationalExceptions 000000000001c29c f   core.obj
 0001:0000b3d8       PollInformationalExceptionsComplete 000000000001c3d8 f   core.obj
 0001:0000b4a4       QueryIOD                   000000000001c4a4 f   himif.obj
 0001:0000b598       QueryCommandComplete       000000000001c598 f   himif.obj
 0001:0000b5d0       XCfgAdapterIF              000000000001c5d0 f   himif.obj
 0001:0000b6ac       PostXCfgAdapterIF          000000000001c6ac f   himif.obj
 0001:0000b900       XlateIODToIOB              000000000001c900 f   himif.obj
 0001:0000ba90       SendToHIM                  000000000001ca90 f   himif.obj
 0001:0000bb58       ReceiveFromHIM             000000000001cb58 f   himif.obj
 0001:0000bd34       IOPull                     000000000001cd34 f   himif.obj
 0001:0000bdb8       DispatchToHIM              000000000001cdb8 f   himif.obj
 0001:0000be60       RetryCommand               000000000001ce60 f   himif.obj
 0001:0000bf00       EnumerateSES2EnclosureDevices 000000000001cf00 f   ses2dev.obj
 0001:0000bf60       DoEnumerateSES2EnclosureDevices 000000000001cf60 f   ses2dev.obj
 0001:0000c3bc       PostSES2ConfigurationDiagPage 000000000001d3bc f   ses2dev.obj
 0001:0000c464       IssueSES2DeviceElementStatusPage 000000000001d464 f   ses2dev.obj
 0001:0000c590       PostSES2DeviceElementStatusPage 000000000001d590 f   ses2dev.obj
 0001:0000c8b8       PostSES2ElementDescriptorPage 000000000001d8b8 f   ses2dev.obj
 0001:0000caa0       AssignDeviceElementNumberToMatchingDevice 000000000001daa0 f   ses2dev.obj
 0001:0000cba4       CdaAssignPTMapForDirectAttachedDevice 000000000001dba4 f   ses2dev.obj
 0001:0000ccf4       CdaAssignPTMapAndNotifyOSM 000000000001dcf4 f   ses2dev.obj
 0001:0000ce08       CoreTimer_CheckIODTimeout  000000000001de08 f   recover.obj
 0001:0000d100       AbortIOD                   000000000001e100 f   recover.obj
 0001:0000d20c       AbortCommandComplete       000000000001e20c f   recover.obj
 0001:0000d2bc       ChannelReset               000000000001e2bc f   recover.obj
 0001:0000d508       PostAbortProbeLuOrDevicePortInitComplete 000000000001e508 f   recover.obj
 0001:0000d508       PostAbortForPACAtAdapterLevel 000000000001e508 f   recover.obj
 0001:0000d544       PostAbortForPACAtPortLevel 000000000001e544 f   recover.obj
 0001:0000d58c       CheckPACForPort            000000000001e58c f   recover.obj
 0001:0000d984       PostResetDevicePortProbeLuOrDevicePortInitComplete 000000000001e984 f   recover.obj
 0001:0000da24       ResetSASHardware           000000000001ea24 f   recover.obj
 0001:0000db38       ResetSASHardwareComplete   000000000001eb38 f   recover.obj
 0001:0000dba8       TimerValidateDevicePort    000000000001eba8 f   recover.obj
 0001:0000dc78       SCSI_MakeSMARTReturnStatusCommand 000000000001ec78 f   ata2scsi.obj
 0001:0000dd40       SCSI_MakeCacheCommand      000000000001ed40 f   ata2scsi.obj
 0001:0000de58       SCSI_MakeSynchronizeCacheCommmand 000000000001ee58 f   ata2scsi.obj
 0001:0000deb8       mv_reset_phy               000000000001eeb8 f   core_adpt.obj
 0001:0000e01c       mv_enable_xmt              000000000001f01c f   core_adpt.obj
 0001:0000e080       Core_GetExpInfo            000000000001f080 f   core_api.obj
 0001:0000e280       Core_MapHDId               000000000001f280 f   core_api.obj
 0001:0000e304       Core_GetHDInformation      000000000001f304 f   core_api.obj
 0001:0000e59c       Core_GetHDInformation_Ext  000000000001f59c f   core_api.obj
 0001:0000e834       Core_GetExpInformationCallback 000000000001f834 f   core_api.obj
 0001:0000e9ec       Core_GetExpInformationHardware 000000000001f9ec f   core_api.obj
 0001:0000eb00       core_pd_request_get_HD_info 000000000001fb00 f   core_api.obj
 0001:0000ebf4       core_pd_request_get_HD_info_ext 000000000001fbf4 f   core_api.obj
 0001:0000ece8       core_pd_request_get_expander_info 000000000001fce8 f   core_api.obj
 0001:0000ed88       core_pd_request_get_HD_config 000000000001fd88 f   core_api.obj
 0001:0000ee74       core_pd_request_get_HD_status 000000000001fe74 f   core_api.obj
 0001:0000ef18       core_pd_request_set_HD_config 000000000001ff18 f   core_api.obj
 0001:0000f198       core_pd_request_BSL_dump   0000000000020198 f   core_api.obj
 0001:0000fed8       Core_InternalSendRequest   0000000000020ed8 f   core_exp.obj
 0001:0000ff5c       HandleInstantRequest       0000000000020f5c f   core_exp.obj
 0001:000102e0       SATA_PrepareCommandHeader  00000000000212e0 f   core_exp.obj
 0001:000103cc       SATA_PrepareCommandTable   00000000000213cc f   core_exp.obj
 0001:000104bc       PrepareDeliveryQueueEntry  00000000000214bc f   core_exp.obj
 0001:00010528       VerifyCommandBeforeSending 0000000000021528 f   core_exp.obj
 0001:000109c4       PrepareAndSendCommand      00000000000219c4 f   core_exp.obj
 0001:00011988       Core_ResetCmdSlot          0000000000022988 f   core_exp.obj
 0001:00011b14       CORE_IssueSMPRequest       0000000000022b14 f   core_exp.obj
 0001:00011c24       SAS_ErrorHandling          0000000000022c24 f   core_exp.obj
 0001:00011ea4       SATA_ErrorHandling         0000000000022ea4 f   core_exp.obj
 0001:000123e4       Port_HandleUnplug          00000000000233e4 f   core_exp.obj
 0001:00012924       Port_Handleplugin          0000000000023924 f   core_exp.obj
 0001:00012da0       SAS_HandleCompletedCommand 0000000000023da0 f   core_exp.obj
 0001:00013878       ServiceInterrupt           0000000000024878 f   core_exp.obj
 0001:0001390c       HandleCommandQueue         000000000002490c f   core_exp.obj
 0001:00013fa8       Core_InterruptServiceRoutine 0000000000024fa8 f   core_exp.obj
 0001:00014004       SATA_HandleDeviceUnplug    0000000000025004 f   core_exp.obj
 0001:00014110       SATA_HandleDevicePlugin    0000000000025110 f   core_exp.obj
 0001:00014278       SATA_PortHandleInterrupt   0000000000025278 f   core_exp.obj
 0001:000148e0       Core_ModuleEnableDisablePHY 00000000000258e0 f   core_extern.obj
 0001:0001495c       Core_FlashRead             000000000002595c f   core_extern.obj
 0001:000149c4       Core_FlashWrite            00000000000259c4 f   core_extern.obj
 0001:00014a34       Core_GetSupportedCounts    0000000000025a34 f   core_helper.obj
 0001:00014ac8       Port_AbortRequests         0000000000025ac8 f   core_helper.obj
 0001:00014db0       Port_IsRequestRunning      0000000000025db0 f   core_helper.obj
 0001:00014e60       GetNCQTag                  0000000000025e60 f   core_helper.obj
 0001:00014efc       MV_DumpRegister            0000000000025efc f   core_helper.obj
 0001:0001505c       FreeDeviceToPool           000000000002605c f   core_helper.obj
 0001:000150e4       GetDeviceFromPool          00000000000260e4 f   core_helper.obj
 0001:00015250       GetExpanderFromPool        0000000000026250 f   core_helper.obj
 0001:0001537c       GetPortFromPool            000000000002637c f   core_helper.obj
 0001:00015480       GetInternalReqFromPool     0000000000026480 f   core_helper.obj
 0001:000154f0       FreeInternalReqToPool      00000000000264f0 f   core_helper.obj
 0001:00015554       GetSATAScratchFromPool     0000000000026554 f   core_helper.obj
 0001:00015590       GetSMPScratchFromPool      0000000000026590 f   core_helper.obj
 0001:000155cc       Expander_SMPReq_Callback   00000000000265cc f   core_helper.obj
 0001:0001571c       Expander_SMPRequest_PhyControl 000000000002671c f   core_helper.obj
 0001:00015820       Expander_SMPRequest_ReportPHYSATA 0000000000026820 f   core_helper.obj
 0001:00015a0c       Device_ATAVoilateRequest   0000000000026a0c f   core_helper.obj
 0001:00015bd0       Device_MakeRequestTaskRequest 0000000000026bd0 f   core_helper.obj
 0001:00015d20       Device_MakeReadCapacityTaskRequest 0000000000026d20 f   core_helper.obj
 0001:00015e10       Device_MakeReadCapacity16TaskRequest 0000000000026e10 f   core_helper.obj
 0001:00015f00       Device_MakeInquiryTaskRequest 0000000000026f00 f   core_helper.obj
 0001:00015fec       Device_MakeReportLunsTaskRequest 0000000000026fec f   core_helper.obj
 0001:000160fc       Device_MakeModeSenseRequest 00000000000270fc f   core_helper.obj
 0001:00016208       FreeRegisterSet            0000000000027208 f   core_helper.obj
 0001:000162cc       AssignRegisterSet          00000000000272cc f   core_helper.obj
 0001:000163a0       mvScsiInquiry              00000000000273a0 f   core_helper.obj
 0001:00016874       mvScsiModeSense            0000000000027874 f   core_helper.obj
 0001:00016c1c       mvScsiReportLun            0000000000027c1c f   core_helper.obj
 0001:00016d00       CheckForDriveFailures      0000000000027d00 f   core_helper.obj
 0001:00016e24       CompleteRequest            0000000000027e24 f   core_helper.obj
 0001:000173d4       CompleteRequestAndSlot     00000000000283d4 f   core_helper.obj
 0001:00017540       HandleDeviceReset          0000000000028540 f   core_helper.obj
 0001:000175f4       HandlePortReset            00000000000285f4 f   core_helper.obj
 0001:0001775c       SATSenseData               000000000002875c f   core_helper.obj
 0001:000178e0       SATSenseData1              00000000000288e0 f   core_helper.obj
 0001:00017a00       RuntimeIssueSoftResetCallback 0000000000028a00 f   core_helper.obj
 0001:00017b0c       RuntimeIssueSoftReset      0000000000028b0c f   core_helper.obj
 0001:00017cbc       RuntimeIssueReadLogExt     0000000000028cbc f   core_helper.obj
 0001:00017dac       RemoveDevice               0000000000028dac f   core_helper.obj
 0001:00017e98       Read_I2C_Register          0000000000028e98 f   core_i2c.obj
 0001:00017edc       Write_I2C_Register         0000000000028edc f   core_i2c.obj
 0001:00017f38       I2C_InterruptServiceRoutine 0000000000028f38 f   core_i2c.obj
 0001:000181e4       I2C_MakeSerialNumber       00000000000291e4 f   core_i2c.obj
 0001:0001834c       I2C_InquiryCmd             000000000002934c f   core_i2c.obj
 0001:00018578       I2C_PrepareAndSendCommand  0000000000029578 f   core_i2c.obj
 0001:0001882c       I2C_IdentifyCallback       000000000002982c f   core_i2c.obj
 0001:00018910       I2C_MakeIdentifyRequest    0000000000029910 f   core_i2c.obj
 0001:00018a0c       CheckI2CDevice             0000000000029a0c f   core_i2c.obj
 0001:00018c4c       FindTgtNo                  0000000000029c4c f   core_ibcd.obj
 0001:00018edc       Issue_ReportGeneral        0000000000029edc f   core_ibcd.obj
 0001:00018f68       Issue_ReportManufacturerInformation 0000000000029f68 f   core_ibcd.obj
 0001:00018ff4       Issue_Discover             0000000000029ff4 f   core_ibcd.obj
 0001:000190e4       Issue_ConfigRouteInfo      000000000002a0e4 f   core_ibcd.obj
 0001:000191e4       DiscoverySM                000000000002a1e4 f   core_ibcd.obj
 0001:00019fc8       DISC_DoDiscover            000000000002afc8 f   core_ibcd.obj
 0001:0001a214       DISC_CancelDiscover        000000000002b214 f   core_ibcd.obj
 0001:0001a2ec       DISC_GetTgtDevMap          000000000002b2ec f   core_ibcd.obj
 0001:0001a3fc       Core_SESExpanderRemove     000000000002b3fc f   core_init.obj
 0001:0001a5cc       SATA_PortDeviceDetected    000000000002b5cc f   core_init.obj
 0001:0001a680       SATA_PortDeviceReady       000000000002b680 f   core_init.obj
 0001:0001a840       SATA_PortReset             000000000002b840 f   core_init.obj
 0001:0001a984       SATA_PortDetect            000000000002b984 f   core_init.obj
 0001:0001aa48       Port_FindTgtNo             000000000002ba48 f   core_init.obj
 0001:0001aae4       CheckDeviceChange          000000000002bae4 f   core_init.obj
 0001:0001acd0       UpdateTargetDevices        000000000002bcd0 f   core_init.obj
 0001:0001af3c       CheckTargetChange          000000000002bf3c f   core_init.obj
 0001:0001b280       UpdateTgtDevMap            000000000002c280 f   core_init.obj
 0001:0001b62c       DiscoveryCallBack          000000000002c62c f   core_init.obj
 0001:0001b744       GetMinNegotiatedLinkRate   000000000002c744 f   core_init.obj
 0001:0001b7a4       GetMaxNegotiatedLinkRate   000000000002c7a4 f   core_init.obj
 0001:0001b804       SAS_PortReset              000000000002c804 f   core_init.obj
 0001:0001bab0       IDSorting                  000000000002cab0 f   core_init.obj
 0001:0001bdfc       I2C_ModuleCheck            000000000002cdfc f   core_init.obj
 0001:0001bec4       mvChannelStateMachine      000000000002cec4 f   core_init.obj
 0001:0001c52c       SATA_DeviceStateMachine0   000000000002d52c f   core_init.obj
 0001:0001c938       SATA_DeviceStateMachine    000000000002d938 f   core_init.obj
 0001:0001cb1c       UpdateWidePortPhyMap       000000000002db1c f   core_init.obj
 0001:0001cd10       DetectPortType             000000000002dd10 f   core_init.obj
 0001:0001cd9c       UpdatePhyInfo              000000000002dd9c f   core_init.obj
 0001:0001d8fc       mvAdapterStateMachine      000000000002e8fc f   core_init.obj
 0001:0001d9b4       CreateDevicesForLus        000000000002e9b4 f   core_init.obj
 0001:0001daec       SAS_Report_LUNs_Data_Changed 000000000002eaec f   core_init.obj
 0001:0001dddc       SAS_InternalReqCallback    000000000002eddc f   core_init.obj
 0001:0001ea20       Port_SoftResetCallback     000000000002fa20 f   core_init.obj
 0001:0001eb18       Device_IssueSoftReset      000000000002fb18 f   core_init.obj
 0001:0001ecd4       Device_ParseIdentifyData   000000000002fcd4 f   core_init.obj
 0001:0001efc8       GetInvernessType           000000000002ffc8 f   core_init.obj
 0001:0001f07c       getSEPDevice               000000000003007c f   core_init.obj
 0001:0001f0b4       SESCmd_CallBack            00000000000300b4 f   core_init.obj
 0001:0001f158       sendRcvDiagRequest         0000000000030158 f   core_init.obj
 0001:0001f214       isPermanentFailure         0000000000030214 f   core_init.obj
 0001:0001f30c       polling_CallBack           000000000003030c f   core_init.obj
 0001:0001f39c       prepareAndSendTestUnitReadyRequest 000000000003039c f   core_init.obj
 0001:0001f470       ReportLUNsDataChange       0000000000030470 f   core_init.obj
 0001:0001f4dc       pollDiagnostics            00000000000304dc f   core_init.obj
 0001:0001f66c       activityBlinker            000000000003066c f   core_init.obj
 0001:0001f720       AssignDeviceElementNumber  0000000000030720 f   core_ses.obj
 0001:0001f850       PostMakeSesElementStatusRequest 0000000000030850 f   core_ses.obj
 0001:0001f92c       PostMakeSesConfigurationRequest 000000000003092c f   core_ses.obj
 0001:0001fa50       PostMakeSesElementDescriptorRequest 0000000000030a50 f   core_ses.obj
 0001:0001fb9c       SES_InternalReqCallback    0000000000030b9c f   core_ses.obj
 0001:0001fc90       Device_MakeSesRcvDiagRequest 0000000000030c90 f   core_ses.obj
 0001:0001fdb4       SGPIO_Initialize           0000000000030db4 f   core_sgpio.obj
 0001:0001ff3c       SGPIOLedStatus             0000000000030f3c f   core_sgpio.obj
 0001:00020080       OdinSPI_WaitDataReady      0000000000031080 f   core_spi.obj
 0001:000200e4       OdinSPI_IssueCmd           00000000000310e4 f   core_spi.obj
 0001:00020158       OdinSPI_PollSR             0000000000031158 f   core_spi.obj
 0001:00020210       OdinSPI_WREN               0000000000031210 f   core_spi.obj
 0001:00020270       OdinSPI_SectErase          0000000000031270 f   core_spi.obj
 0001:000202e8       OdinSPI_WriteBuf           00000000000312e8 f   core_spi.obj
 0001:000203d4       OdinSPI_Read               00000000000313d4 f   core_spi.obj
 0001:00020464       OdinSPI_ReadBuf            0000000000031464 f   core_spi.obj
 0001:00020538       OdinSPI_Init               0000000000031538 f   core_spi.obj
 0001:00020630       Category_CDB_Type          0000000000031630 f   scsi2sata.obj
 0001:000207ec       SCSI_ATA_EnableDisableFeature 00000000000317ec f   scsi2sata.obj
 0001:0002088c       SCSI_ATA_InquiryTranslationCallback 000000000003188c f   scsi2sata.obj
 0001:00020cac       SCSI_ATA_LogSenseTranslation 0000000000031cac f   scsi2sata.obj
 0001:00020d7c       SCSI_ATA_ModeSenseTranslation 0000000000031d7c f   scsi2sata.obj
 0001:00020efc       SCSI_ATA_ModeSelectTranslation 0000000000031efc f   scsi2sata.obj
 0001:00021020       SCSI_ATA_ReadWriteTranslation 0000000000032020 f   scsi2sata.obj
 0001:00021124       SCSI_ATA_ReadCapacityTranslationCallback 0000000000032124 f   scsi2sata.obj
 0001:00021170       SCSI_ATA_TestUnitReadyTranslationCallback 0000000000032170 f   scsi2sata.obj
 0001:000211a4       ATA_CDB2TaskFile           00000000000321a4 f   scsi2sata.obj
 0001:00021718       ATAPI_CDB2TaskFile         0000000000032718 f   scsi2sata.obj
 0001:00021844       Tag_Init                   0000000000032844 f   com_tag.obj
 0001:00021880       MV_DecodeReadWriteCDB      0000000000032880 f   com_util.obj
 0001:00021a28       MvCreateInitializationTSCB 0000000000032a28 f   mvchim_init.obj
 0001:00021b38       MvGetConfiguration         0000000000032b38 f   mvchim_init.obj
 0001:00021b58       MvAdjustLuProfile          0000000000032b58 f   mvchim_utils.obj
 0001:00021b58       MvAdjustPhyProfile         0000000000032b58 f   mvchim_utils.obj
 0001:00021b58       MvSetConfiguration         0000000000032b58 f   mvchim_init.obj
 0001:00021b58       MvAdjustPortProfile        0000000000032b58 f   mvchim_utils.obj
 0001:00021b58       MvPollIRQ                  0000000000032b58 f   mvchim_utils.obj
 0001:00021b58       MvAdjustDevicePortProfile  0000000000032b58 f   mvchim_utils.obj
 0001:00021b58       MvClearLuTSH               0000000000032b58 f   mvchim_utils.obj
 0001:00021b58       MvCheckIOBMemoryNeeded     0000000000032b58 f   mvchim_init.obj
 0001:00021b58       MvDeleteAdapterTSCB        0000000000032b58 f   mvchim_init.obj
 0001:00021b64       MvSizeAdapterTSCB          0000000000032b64 f   mvchim_init.obj
 0001:00021b70       MvCreateAdapterTSCB        0000000000032b70 f   mvchim_init.obj
 0001:00021c0c       MvSetupAdapterTSCB         0000000000032c0c f   mvchim_init.obj
 0001:00021c2c       MvCheckMemoryNeeded        0000000000032c2c f   mvchim_init.obj
 0001:00021cd8       MvSetMemoryPointer         0000000000032cd8 f   mvchim_init.obj
 0001:00021f20       MvVerifyAdapter            0000000000032f20 f   mvchim_init.obj
 0001:00021f88       mv_init                    0000000000032f88 f   mvchim_init.obj
 0001:0002208c       MvGetPhyTSH                000000000003308c f   mvchim_init.obj
 0001:00022110       MvFrontEndISR              0000000000033110 f   mvchim_init.obj
 0001:0002213c       MvGetPortTSH               000000000003313c f   mvchim_init.obj
 0001:00022180       MvSizeDevicePortTSCB       0000000000033180 f   mvchim_init.obj
 0001:0002218c       MvQueueIOB                 000000000003318c f   mvchim_init.obj
 0001:000227a8       update_tscbs_frm_core      00000000000337a8 f   mvchim_init.obj
 0001:00022884       MvCheckDevPortTSCBNeeded   0000000000033884 f   mvchim_init.obj
 0001:0002293c       MvCreateDevicePortTSCB     000000000003393c f   mvchim_init.obj
 0001:00022a40       MvValidateDevicePortTSH    0000000000033a40 f   mvchim_init.obj
 0001:00022b5c       MvValidatePortTSH          0000000000033b5c f   mvchim_init.obj
 0001:00022b80       MvClearDevicePortTSH       0000000000033b80 f   mvchim_init.obj
 0001:00022ba0       MvClearPortTSH             0000000000033ba0 f   mvchim_init.obj
 0001:00022bc0       MvSizeLuTSCB               0000000000033bc0 f   mvchim_init.obj
 0001:00022bcc       MvCreateLuTSCB             0000000000033bcc f   mvchim_init.obj
 0001:00022bf0       MvCheckDeviceStatus        0000000000033bf0 f   mvchim_init.obj
 0001:00022c24       MvCheckReportLUNSDataChange 0000000000033c24 f   mvchim_init.obj
 0001:00022c58       copy_frm_iob_sg            0000000000033c58 f   mvchim_utils.obj
 0001:00022cc0       HBA_Notification           0000000000033cc0 f   mvchim_utils.obj
 0001:00022e18       MvBackEndISR               0000000000033e18 f   mvchim_init.obj
 0001:00022e18       MvDisableIRQ               0000000000033e18 f   mvchim_init.obj
 0001:00022e18       OSMSynchronizeRange        0000000000033e18 f   osmif.obj
 0001:00022e18       MvEnableIRQ                0000000000033e18 f   mvchim_init.obj
 0001:00022e18       OSMWatchdog                0000000000033e18 f   osmif.obj
 0001:00022e18       HBARequestCallback         0000000000033e18 f   mvchim_utils.obj
 0001:00022e24       MvWriteNVSegment           0000000000033e24 f   mvchim_utils.obj
 0001:00022e5c       MvReadNVSegment            0000000000033e5c f   mvchim_utils.obj
 0001:00022ea8       MvReadRAMSegment           0000000000033ea8 f   mvchim_utils.obj
 0001:00022ef0       MvWriteRAMSegment          0000000000033ef0 f   mvchim_utils.obj
 0001:00022f28       MvSectEraseRAMSegment      0000000000033f28 f   mvchim_utils.obj
 0001:00022fac       MvProfileAdapter           0000000000033fac f   mvchim_utils.obj
 0001:00022fcc       MvAdjustAdapterProfile     0000000000033fcc f   mvchim_utils.obj
 0001:00022fe0       MvProfilePort              0000000000033fe0 f   mvchim_utils.obj
 0001:00022ff4       MvProfileDevicePort        0000000000033ff4 f   mvchim_utils.obj
 0001:00023120       MvProfilePhy               0000000000034120 f   mvchim_utils.obj
 0001:00023134       MvProfileLu                0000000000034134 f   mvchim_utils.obj
 0001:00023154       MvInitialize               0000000000034154 f   mvchim_utils.obj
 0001:00023200       MVOSMReadUExact32          0000000000034200 f   mvchim_utils.obj
 0001:00023258       MVOSMWriteUExact32         0000000000034258 f   mvchim_utils.obj
 0001:000232c0       res_get_req_from_pool      00000000000342c0 f   res_mgmt.obj
 0001:00023390       __security_check_cookie    0000000000034390 f   BufferOverflowK:amdsecgs.obj
 0001:000233b8       __report_gsfailure         00000000000343b8 f   BufferOverflowK:gs_report.obj
 0001:000233f0       memcpy                     00000000000343f0 f   storport:memcpy.obj
 0001:000233f0       memmove                    00000000000343f0     storport:memcpy.obj
 0001:00023740       memset                     0000000000034740 f   storport:memset.obj
 0001:00023830       __GSHandlerCheckCommon     0000000000034830 f   sehupd:gshandler.obj
 0001:0002389c       __GSHandlerCheck           000000000003489c f   sehupd:gshandler.obj
 0001:000238c0       ??_C@_06KGPGLGBE@dump?$DN1?$AA@FNODOBFM@ 00000000000348c0     regreader.obj
 0001:000238d0       ??_C@_07HPMHGBON@ntldr?$DN1?$AA@FNODOBFM@ 00000000000348d0     regreader.obj
 0001:000238e0       ??_C@_1CG@GDNLFIP@?$AA?2?$AAP?$AAa?$AAr?$AAa?$AAm?$AAe?$AAt?$AAe?$AAr?$AAs?$AA?2?$AAD?$AAe?$AAv?$AAi?$AAc?$AAe?$AA?$AA@FNODOBFM@ 00000000000348e0     regreader.obj
 0001:00023910       ??_C@_1BM@JEGNIDLI@?$AAM?$AAa?$AAx?$AAi?$AAm?$AAu?$AAm?$AAS?$AAG?$AAL?$AAi?$AAs?$AAt?$AA?$AA@FNODOBFM@ 0000000000034910     regreader.obj
 0001:00023930       ??_C@_1BA@MHCBCPNL@?$AAM?$AAa?$AAx?$AAT?$AAa?$AAg?$AAs?$AA?$AA@FNODOBFM@ 0000000000034930     regreader.obj
 0001:00023940       ??_C@_1BA@CMKGIANO@?$AAM?$AAa?$AAx?$AAL?$AAu?$AAn?$AAs?$AA?$AA@FNODOBFM@ 0000000000034940     regreader.obj
 0001:00023950       ??_C@_08PABONNMM@wakeup?$DN1?$AA@FNODOBFM@ 0000000000034950     ntinit.obj
 0001:00023960       ??_C@_0M@DCLFAKAJ@HBA?5?5?5?5?5?5?5?5?$AA@FNODOBFM@ 0000000000034960     ntinit.obj
 0001:00023970       ??_C@_06EDFEKNLJ@MVSATA?$AA@FNODOBFM@ 0000000000034970     core_helper.obj
 0001:00023980       ??_C@_0BB@JCEFLFJE@0123456789abcdef?$AA@FNODOBFM@ 0000000000034980     core_i2c.obj
 0002:00000000       __imp_RtlQueryRegistryValues 0000000000035000     wdm:NTOSKRNL.exe
 0002:00000008       __imp_RtlInitUnicodeString 0000000000035008     wdm:NTOSKRNL.exe
 0002:00000010       __imp_ExAllocatePoolWithTag 0000000000035010     wdm:NTOSKRNL.exe
 0002:00000018       __imp_IoAllocateErrorLogEntry 0000000000035018     wdm:NTOSKRNL.exe
 0002:00000020       __imp_IoWriteErrorLogEntry 0000000000035020     wdm:NTOSKRNL.exe
 0002:00000028       __imp_KeBugCheckEx         0000000000035028     storport:NTOSKRNL.exe
 0002:00000030       \177NTOSKRNL_NULL_THUNK_DATA 0000000000035030     storport:NTOSKRNL.exe
 0002:00000038       __imp_StorPortReady        0000000000035038     storport:storport.sys
 0002:00000040       __imp_StorPortGetUncachedExtension 0000000000035040     storport:storport.sys
 0002:00000048       __imp_StorPortInitialize   0000000000035048     storport:storport.sys
 0002:00000050       __imp_StorPortStallExecution 0000000000035050     storport:storport.sys
 0002:00000058       __imp_StorPortGetPhysicalAddress 0000000000035058     storport:storport.sys
 0002:00000060       __imp_StorPortGetLogicalUnit 0000000000035060     storport:storport.sys
 0002:00000068       __imp_StorPortLogError     0000000000035068     storport:storport.sys
 0002:00000070       __imp_StorPortBusy         0000000000035070     storport:storport.sys
 0002:00000078       __imp_StorPortResumeDevice 0000000000035078     storport:storport.sys
 0002:00000080       __imp_StorPortSetDeviceQueueDepth 0000000000035080     storport:storport.sys
 0002:00000088       __imp_StorPortGetDeviceBase 0000000000035088     storport:storport.sys
 0002:00000090       __imp_StorPortPauseDevice  0000000000035090     storport:storport.sys
 0002:00000098       __imp_StorPortGetBusData   0000000000035098     storport:storport.sys
 0002:000000a0       __imp_StorPortSetBusDataByOffset 00000000000350a0     storport:storport.sys
 0002:000000a8       __imp_StorPortNotification 00000000000350a8     storport:storport.sys
 0002:000000b0       \177storport_NULL_THUNK_DATA 00000000000350b0     storport:storport.sys
 0003:00000000       HotPatchBuffer             0000000000036000     hotpatch.obj
 0003:00000100       __security_cookie          0000000000036100     BufferOverflowK:gs_support.obj
 0003:00000108       __security_cookie_complement 0000000000036108     BufferOverflowK:gs_support.obj
 0003:00000110       MvFuncPtrs                 0000000000036110     mvchim_init.obj
 0003:000002c0       MVConfiguration            00000000000362c0     mvchim_init.obj
 0003:00000338       I2C_INQUIRY_DEVICE_DATA    0000000000036338     core_i2c.obj
 0003:0000035c       I2C_INQUIRY_VPD_PAGE80_DATA 000000000003635c     core_i2c.obj
 0003:00000760       ATMEL_SPI_CMD              0000000000036760     core_spi.obj
 0003:00000770       MXIC_SPI_CMD               0000000000036770     core_spi.obj
 0003:00000780       I2C_INQUIRY_VPD_PAGE0_DATA 0000000000036780     core_i2c.obj
 0003:00000788       I2C_INQUIRY_VPD_PAGE83_DATA 0000000000036788     core_i2c.obj
 0003:00000820       __core_mod_ops             0000000000036820     core_exp.obj
 0003:00000880       core_pd_cmd_handler        0000000000036880     core_api.obj
 0003:000008d0       ChipsSupported             00000000000368d0     ntinit.obj
 0003:00000904       Global_Eip_Bit             0000000000036904     ses2dev.obj
 0003:00000905       Enclosure_Flag             0000000000036905     ses2dev.obj
 0003:00000907       Discovery_state            0000000000036907     core_ibcd.obj
 0003:00000918       modePageBuf                0000000000036918     scsi2sata.obj
 0003:00000934       temp                       0000000000036934     <common>
 0003:00000938       driverObjectRef            0000000000036938     <common>
 0003:00000940       stopadapter_called         0000000000036940     <common>
 0003:00000960       regPath                    0000000000036960     <common>
 0003:00000b5e       max_io                     0000000000036b5e     <common>
 0005:00000008       GsDriverEntry              0000000000038008 f   BufferOverflowK:gs_support.obj
 0005:00000064       __IMPORT_DESCRIPTOR_storport 0000000000038064     storport:storport.sys
 0005:00000078       __IMPORT_DESCRIPTOR_NTOSKRNL 0000000000038078     storport:NTOSKRNL.exe
 0005:0000008c       __NULL_IMPORT_DESCRIPTOR   000000000003808c     storport:NTOSKRNL.exe

 entry point at        0005:00000008

 Static symbols

 0001:0000f1a8       mv_is_sig_fis_received     00000000000201a8 f    CIL library: CIL module
 0001:0000f23c       __core_ops_get_res_desc    000000000002023c f    CIL library: CIL module
 0001:0000f484       __core_ops_init            0000000000020484 f    CIL library: CIL module
 0001:0000fde4       __core_ops_start           0000000000020de4 f    CIL library: CIL module
 0001:0000fe00       __core_ops_stop            0000000000020e00 f    CIL library: CIL module
 0001:0000ff50       __core_ops_send_request    0000000000020f50 f    CIL library: CIL module
 0001:00011a4c       IBCD_SMPReq_Callback       0000000000022a4c f    CIL library: CIL module
 0001:00012104       __handle_waiting_list      0000000000023104 f    CIL library: CIL module
 0001:00012ac4       Port_HandlePortInterrupt   0000000000023ac4 f    CIL library: CIL module
 0001:00014858       __core_ops_monitor         0000000000025858 f    CIL library: CIL module
 0001:00014884       __core_ops_reset           0000000000025884 f    CIL library: CIL module
 0001:000158e8       Core_TaskReqCallback       00000000000268e8 f    CIL library: CIL module
 0001:00015af0       Core_ATASetFeatureReqCallback 0000000000026af0 f    CIL library: CIL module
 0001:00016a50       modeSelect                 0000000000027a50 f    CIL library: CIL module
 0001:00017b9c       RuntimeIssueReqCallback    0000000000028b9c f    CIL library: CIL module
 0001:00018cbc       SMP_Callback               0000000000029cbc f    CIL library: CIL module
 0001:0001c260       SAS_DeviceStateMachine     000000000002d260 f    CIL library: CIL module
 0001:0001c9ac       ResetController            000000000002d9ac f    CIL library: CIL module
 0001:0001d0dc       InitChip                   000000000002e0dc f    CIL library: CIL module
 0001:0001e700       SATA_InternalReqCallback   000000000002f700 f    CIL library: CIL module
 0001:0001ebd0       Device_IssueIdentify       000000000002fbd0 f    CIL library: CIL module
 0001:000226d0       MvQueueIOB_Callback        00000000000336d0 f    CIL library: CIL module
